:10000000370101002920A94873000000828052B8FE
:1000100037440F001304F4230145A2858D282120C5
:1000200029451128D5BF854873000000828091487A
:10003000730000008280AD48730000008280930846
:1000400010087300000082809308500873000000BD
:10005000828093087008730000008280732510C0AE
:100060008280732500C082809308600873000000BE
:1000700082800589F322008093920248B3E2A200B5
:1000800073900280828095487300000082809308FC
:100090000008730000008280A14873000000828085
:1000A00093083008730000008280930840087300B2
:0400B000000082804A
:00000001FF
